:100000008312850186010528492981018316F03074
:100010008500FF3086005F3081008312A0308B00A6
:10002000930125308C00DC2006308D000321C62092
:100030003F21C6200621C6201A21C6204221C62003
:100040002521C620C620C6202521C620AD20C620D9
:100050000F21C6203C21C6200821C6201521C6201C
:10006000C620C6200030F7208C00DC200130F720AD
:10007000A2000F398D00220E0F398E000230F720BA
:10008000A2000F399100220E0F398F000330F720A4
:1000900090000430F720E03903195128E03C031D9B
:1000A0005C2815308C00DC20AD20C6204221C62003
:1000B000422102306D2154280E086D211108920052
:1000C00003309E0001309F00A1018E20A10D8E20E3
:1000D000A10D8E20A10DA108031981289319812853
:1000E0000730210203197E288E20031C7928B220B4
:1000F0007A28AD20A10B7428C6206428C620C6200B
:100100006428920303198728C620C62060280F0898
:100110006D21A52010086D21A9205C2803109F0CDB
:10012000031C9E2880309F009E0A40301E02031C44
:100130009B28931508001E08F720A0001F08200523
:1001400003190310031D0314080005148515131566
:1001500008000510851113110800A520B720A9205B
:10016000B7200800A520C620A920B7200800140841
:1001700097001508980016089900980A990A970B95
:10018000BF28980BBF28990BBF28080014089A00B5
:1001900015089B0016089C000310960C950C940CF7
:1001A0000D089D00B7209D0BD2281A0894001B084B
:1001B00095001C08960008000C08AE002F30AB001C
:1001C0009130AC000530AD00AF01950196010130D2
:1001D0009400AB0DAC0DAD0DAF0D2E082F02031822
:1001E000AF00940D950D960D031CE92808008312AD
:1001F000890083168B130814831208088B170800D4
:10020000AD20AD20AD20AD20AD200800B220B22041
:10021000B220B220B2200800AD20AD20AD20AD202C
:10022000B2200800B220B220B220B220AD200800D7
:10023000AD20AD20AD20B220B2200800B220B22007
:10024000B220AD20AD200800B220B220AD20AD20FC
:10025000AD200800AD20AD20B220B220B2200800B1
:10026000B220AD20AD20AD20AD200800AD20B220E1
:10027000B220B220B2200800152115210800152156
:10028000B2200800AD20B220AD200800B2201A2113
:100290000800A300030EA4000B11A90A0319AA0A5F
:1002A0000F302A02031C5B2942302902031C5B2900
:1002B000A901AA01A80A131D6629931C632993109A
:1002C0008510051566299314051185148B168B1757
:1002D000240E8300A30E230E0900A200A901AA0187
:0C02E000A80128082202031D7129080053
:02400E00F13F80
:104200001000260021000F0089002E009E004300B0
:10421000EE00D9004800EE00BF004F0042009800B9
:10422000E0000000000000000000000000000000AE
:10423000000000000000000000000000000000007E
:10424000000000000000000000000000000000006E
:10425000000000000000000000000000000000005E
:10426000000000000000000000000000000000004E
:10427000000000000000000000000000000000003E
:00000001FF
